:020000040000FA
:04000000DD303A288D
:08000800A000030EA100831209
:1000100005191028831601178312B23081002B288E
:1000200083160113831203140B190310A80DA90DD5
:10003000AA0DAB0DAC0DAC16FF302C02031D2B2806
:10004000FA302B02031D2B2831152A08AF0029088E
:10005000AE002808AD008B100B11210E8300A00EFE
:04006000200E090065
:0C007400203084008001840A80300402E7
:10008000031C3C281230B0007F2183160C308505FC
:1000900087018312850187010730990000309A009B
:1000A000103083168E008312603083168F00831207
:1000B0000030831691009F008312C83083168100A0
:1000C000831231309000003083168C008312103080
:1000D0008B00831610309B001C141A088312BD007D
:1000E000332281018E018F010B118B100B108C01BB
:1000F0008B17892031198C206121B30B87280310BD
:1001000085190314B90DF030390203190A2144226C
:10011000792864003210080031110130B7008B13C8
:100120002030370783169B001C141A088312A40082
:100130001030370783169B001C141A088312A30083
:10014000A6000230A6060030370783169B001C1459
:100150001A088312A200A7000130A7068B17321CD1
:10016000B72822090339A200A309A409A509240874
:100170002F02031D042923082E02031DDF28220855
:100180002D02031D042901303702031DCA283D1426
:100190003E14872102303702031DD128BD143E14BE
:1001A0009D2103303702031DD8283D153E14B3218D
:1001B00004303702031DDF28BD153E14C92126086F
:1001C0002E02031D042927082D02031D04290130D6
:1001D0003702031DEE283D103E14DF2102303702A6
:1001E000031DF528BD103E14F42103303702031D12
:1001F000FC283D113E14092204303702031D032957
:10020000BD113E141E220429B70A05303702031817
:1002100008008F280130B600B300B400B500B70065
:1002200085018701B1138920B30B3029031085198B
:100230000314B90DF030390203195729B41F850191
:10024000B41F8701B40B30293708B6080319B6006C
:1002500003192E29FF3085008700B6039630B400BD
:10026000311D13293111321C3A292D090339AD00F2
:10027000AE09AF092F1C13298E018F010C1C132905
:100280000C102E1E13298B1320303707BB002F08AC
:10029000BA006A2110303707BB002E08BA006A2165
:1002A00000303707BB002D08BA006A218B17850183
:1002B0008701B70AB60105303702031C1329332220
:1002C00008003E1C08003E101030BB003D08BA007C
:1002D0006A2108008B133A0883161C159A008312B2
:1002E0003B0883169B0055309D00AA309D009C144E
:1002F00064009C1878291C1183128B170800831640
:1003000010309B001C141A088312BD0008003D1415
:100310006430D5005D27E0006730D5005D27E1003F
:100320006530D5005D27C4006630D5005D27CC0060
:100330000130C800FF30C0000800BD146430D50093
:100340006727E2006730D5006727E3006530D500F6
:100350006727C5006630D5006727CD000130C9008A
:10036000FF30C10008003D156430D5007127E4005E
:100370006730D5007127E5006530D5007127C600CC
:100380006630D5007127CE000130CA00FF30C200B0
:100390000800BD156430D5007B27E6006730D50026
:1003A0007B27E7006530D5007B27C7006630D50086
:1003B0007B27CF000130CB00FF30C3000800601A5C
:1003C0000512E01A8512601B0510E01B85106118EC
:1003D0008710E118071161190710E1198712611AD6
:1003E0000712E11A87110800621A0512E21A851233
:1003F000621B0510E21B851063188710E3180711B4
:1004000063190710E3198712631A0712E31A871199
:100410000800641A0512E41A8512641B0510E41B17
:10042000851065188710E518071165190710E5197B
:100430008712651A0712E51A87110800661A051255
:10044000E61A8512661B0510E61B851067188710D3
:10045000E718071167190710E7198712671A0712BB
:10046000E71A871108003D188721601C3D10BD1850
:100470009D21621CBD103D19B321641C3D11BD19A5
:10048000C921661CBD110800D001D01B8721501B5B
:100490009D21D01AB321501AC9210A300F02031C22
:1004A00008008E018F013D1C702AC80B702A4C0871
:1004B000C800C00A4408400203186C2A4008D5004E
:1004C0005D27D0004008D5006227D1006008E80011
:1004D0006108E9002027702AC00160185E2A3D10DB
:1004E000BD1C8D2AC90B8D2A4D08C900C10A4508BB
:1004F00041020318892A4108D5006727D000410826
:10050000D5006C27D1006208E8006308E9002027C5
:100510008D2AC10162187B2ABD103D1DAA2ACA0B73
:10052000AA2A4E08CA00C20A460842020318A62A8E
:100530004208D5007127D0004208D5007627D100A7
:100540006408E8006508E9002027AA2AC2016418A7
:10055000982A3D11BD1DC72ACB0BC72A4F08CB00D7
:10056000C30A470843020318C32A4308D5007B2760
:10057000D0004308D5008027D1006608E80067084E
:10058000E9002027C72AC3016618B52ABD11080053
:10060000003401340234033404340534063407342E
:10061000083409340A340B340C340D340E340F34DE
:10062000103411341234133414341534163417348E
:10063000183419341A341B341C341D341E341F343E
:1006400020342134223423342434253426342734EE
:10065000283429342A342B342C342D342E342F349E
:10066000303431343234333434343534363437344E
:10067000383439343A343B343C343D343E343F34FE
:1006800040344134423443344434453446344734AE
:10069000483449344A344B344C344D344E344F345E
:1006A000503451345234533454345534563457340E
:1006B000583459345A345B345C345D345E345F34BE
:1006C0006034613462346334F13464341E343F3452
:1006D000003400340034003400340034003400347A
:1006E000003400340034003400340034003400346A
:1006F000003400340034003400340034003400345A
:10070000003401340234033404340534063407342D
:10071000083409340A340B340C340D340E340F34DD
:10072000103411341234133414341534163417348D
:10073000183419341A341B341C341D341E341F343D
:1007400020342134223423342434253426342734ED
:10075000283429342A342B342C342D342E342F349D
:10076000303431343234333434343534363437344D
:10077000383439343A343B343C343D343E343F34FD
:1007800040344134423443344434453446344734AD
:10079000483449344A344B344C344D344E344F345D
:1007A000503451345234533454345534563457340D
:1007B000583459345A345B345C345D345E345F34BD
:1007C0006034613462346334003400340034003403
:1007D0000034003400340034003400340034003479
:1007E0000034003400340034003400340034003469
:1007F0000034003400340034003400340034003459
:10080000003401340234033404340534063407342C
:10081000083409340A340B340C340D340E340F34DC
:10082000103411341234133414341534163417348C
:10083000183419341A341B341C341D341E341F343C
:1008400020342134223423342434253426342734EC
:10085000283429342A342B342C342D342E342F349C
:10086000303431343234333434343534363437344C
:10087000383439343A343B343C343D343E343F34FC
:1008800040344134423443344434453446344734AC
:10089000483449344A344B344C344D344E344F345C
:1008A000503451345234533454345534563457340C
:1008B000583459345A345B345C345D345E345F34BC
:1008C0006034613462346334F13464341E343F3450
:1008D0000034003400340034003400340034003478
:1008E0000034003400340034003400340034003468
:1008F0000034003400340034003400340034003458
:10090000003401340234033404340534063407342B
:10091000083409340A340B340C340D340E340F34DB
:10092000103411341234133414341534163417348B
:10093000183419341A341B341C341D341E341F343B
:1009400020342134223423342434253426342734EB
:10095000283429342A342B342C342D342E342F349B
:10096000303431343234333434343534363437344B
:10097000383439343A343B343C343D343E343F34FB
:1009800040344134423443344434453446344734AB
:10099000483449344A344B344C344D344E344F345B
:1009A000503451345234533454345534563457340B
:1009B000583459345A345B345C345D345E345F34BB
:1009C0006034613462346334003400340034003401
:1009D0000034003400340034003400340034003477
:1009E0000034003400340034003400340034003467
:1009F0000034003400340034003400340034003457
:100A0000003401340234033404340534063407342A
:100A1000083409340A340B340C340D340E340F34DA
:100A2000103411341234133414341534163417348A
:100A3000183419341A341B341C341D341E341F343A
:100A400020342134223423342434253426342734EA
:100A5000283429342A342B342C342D342E342F349A
:100A6000303431343234333434343534363437344A
:100A7000383439343A343B343C343D343E343F34FA
:100A800040344134423443344434453446344734AA
:100A9000483449344A344B344C344D344E344F345A
:100AA000503451345234533454345534563457340A
:100AB000583459345A345B345C345D345E345F34BA
:100AC0006034613462346334F13464341E343F344E
:100AD0000034003400340034003400340034003476
:100AE0000034003400340034003400340034003466
:100AF0000034003400340034003400340034003456
:100B00000034013402340334043405340634073429
:100B1000083409340A340B340C340D340E340F34D9
:100B20001034113412341334143415341634173489
:100B3000183419341A341B341C341D341E341F3439
:100B400020342134223423342434253426342734E9
:100B5000283429342A342B342C342D342E342F3499
:100B60003034313432343334343435343634373449
:100B7000383439343A343B343C343D343E343F34F9
:100B800040344134423443344434453446344734A9
:100B9000483449344A344B344C344D344E344F3459
:100BA0005034513452345334543455345634573409
:100BB000583459345A345B345C345D345E345F34B9
:100BC00060346134623463340034003400340034FF
:100BD0000034003400340034003400340034003475
:100BE0000034003400340034003400340034003465
:100BF0000034003400340034003400340034003455
:100C00000034013402340334043405340634073428
:100C1000083409340A340B340C340D340E340F34D8
:100C20001034113412341334143415341634173488
:100C3000183419341A341B341C341D341E341F3438
:100C400020342134223423342434253426342734E8
:100C5000283429342A342B342C342D342E342F3498
:100C60003034313432343334343435343634373448
:100C7000383439343A343B343C343D343E343F34F8
:100C800040344134423443344434453446344734A8
:100C9000483449344A344B344C344D344E344F3458
:100CA0005034513452345334543455345634573408
:100CB000583459345A345B345C345D345E345F34B8
:100CC0006034613462346334F13464341E343F344C
:100CD0000034003400340034003400340034003474
:100CE0000034003400340034003400340034003464
:100CF0000034003400340034003400340034003454
:100D00000034013402340334043405340634073427
:100D1000083409340A340B340C340D340E340F34D7
:100D20001034113412341334143415341634173487
:100D3000183419341A341B341C341D341E341F3437
:100D400020342134223423342434253426342734E7
:100D5000283429342A342B342C342D342E342F3497
:100D60003034313432343334343435343634373447
:100D7000383439343A343B343C343D343E343F34F7
:100D800040344134423443344434453446344734A7
:100D9000483449344A344B344C344D344E344F3457
:100DA0005034513452345334543455345634573407
:100DB000583459345A345B345C345D345E345F34B7
:100DC00060346134623463340034003400340034FD
:100DD0000034003400340034003400340034003473
:100DE0000034003400340034003400340034003463
:100DF0000034003400340034003400340034003453
:100E4000681E262F501C051250180516E81E2C2F60
:100E5000D01C8512D0188516681F322F501D051022
:100E600050190514E81F382FD01D8510D01985148E
:100E7000691C3E2F511C871051188714E91C442F00
:100E8000D11C0711D1180715691D4A2F511D0710D4
:100E900051190714E91D502FD11D8712D11987163A
:100EA000691E562F511E0712511A0716E91E5C2F94
:100EB000D11E8711D11A8715080003308A00D51377
:100EC0005508820003308A00D51755088200043087
:100ED0008A00D5135508820004308A00D5175508BA
:100EE000820005308A00D5135508820005308A003B
:100EF000D5175508820006308A00D51355088200A0
:0A0F000006308A00D517550882005C
:084000000F000300050003009E
:02400E00CC33B1
:10420000010078007A007C007E007B0079007F004E
:104210007D007A0078007E007C00FF00FF00FF0038
:104220000000F200F600FA00FE00F200F600FA00CC
:10423000FE00F200F600FA00FE00FF00FF00FF00A3
:10424000010005000500050005000900090009003E
:1042500009000D000D000D000D00FF00FF00FF0024
:10426000FF00FF00FF00FF00FF00FF00FF00FF0056
:10427000FF00FF00FF00FF00FF00FF00FF00FF0046
:10428000FF00FF00FF00FF00FF00FF00FF00FF0036
:10429000FF00FF00FF00FF00FF00FF00FF00FF0026
:1042A000FF00FF00FF00FF00FF00FF00FF00FF0016
:1042B000FF00FF00FF00FF00FF00FF00FF00FF0006
:1042C000FF00FF00FF00FF00FF00FF00FF00FF00F6
:1042D000FF00FF00FF00FF00FF00FF00FF00FF00E6
:1042E000FF00FF00FF00FF00FF00FF00FF00FF00D6
:1042F000FF00FF00FF00FF00FF00FF00FF00DD00E8
:00000001FF
